:060000000A128A11CA2D4C
:100B9400F001F101F201F301F401F501F601F701AD
:100BA400A001A10183010A128A11542EFA00E42D36
:100BB400F230F8000130F9000A128A11EC250A1209
:100BC4008A11E42D0130FA02031DE92DEA2DDA2DF4
:100BD400EB2D0800F001F101F82D000000000000E9
:100BE4000130F0070318F10A0030F10779087106A3
:100BF400031DFE2D78087006031D012E022EEF2D15
:100C0400032E08004B30FA007A08FB00242E8312CE
:100C14000313871207167B30F8000030F9000A121C
:100C24008A11EC250A128A118312031307128716FC
:100C34007B30F8000030F9000A128A11EC250A1200
:100C44008A11242E0130FB02031D292E2A2E092E7F
:100C54002B2E08009630FA007A08FB004C2E8312E3
:100C64000313871207163D30F8000030F9000A120A
:100C74008A11EC250A128A118312031307128716AC
:100C84003D30F8000030F9000A128A11EC250A12EE
:100C94008A114C2E0130FB02031D512E522E312E8F
:100CA400532E08008B010730831603139C00063073
:100CB4009F0085108B01EF30860083120313061604
:100CC4008B01CF308316031387000030F700F60042
:100CD400F500F400F300FC007C08F200712E0A1207
:100CE4008A1111270A128A11FC007C08FD007D0874
:100CF400013A031D7E2E7F2E832E831203130612C8
:100D0400712E7D08023A031D882E892E8D2E8312A2
:100D140003130616712E7D08033A031D922E932E9B
:100D2400972E831203138514712E7D08043A031D34
:100D34009C2E9D2EA12E831203138510712E7D08E7
:100D4400053A031DA62EA72EAD2E0A128A112C26B3
:100D54000A128A11712E7D08063A031DB22EB32E93
:100D6400B92E0A128A1104260A128A11712E7D08DC
:100D7400073A031DBE2EBF2EC52E0A128A112C2639
:100D84000A128A11712E7D08083A031DCA2ECB2E31
:100D9400D12E0A128A1104260A128A11712E7D0894
:100DA400093A031DD62ED72EDD2E0A128A112C26BF
:100DB4000A128A11712E7D080A3A031DE22EE32ECF
:100DC400E92E0A128A1104260A128A11712E7D084C
:100DD4000B3A031DEE2EEF2EF52E0A128A112C2645
:100DE4000A128A11712E7D080C3A031DFA2EFB2E6D
:100DF400712E0A128A1104260A128A11712E712E7A
:100E0400712E712E712E712E712E712E712E712EE6
:100E1400712E712E712E712E0A128A11002807303C
:100E2400FB007B088312031386040730FB007B0856
:100E3400831603138604FE30FB007B08860502300C
:100E44000A128A11D8250A128A1183120313861CE6
:100E54002C2F2D2F372FF208031D312F322F372F30
:100E6400F201F20A0130FF2FFF2F86183A2F3B2F91
:100E7400452F7208013A031D402F412F452FF201DF
:100E84000230FF2FFF2F061D482F492F532FF7083D
:100E9400031D4D2F4E2F532FF701F70A0B30FF2F51
:100EA400FF2F0619562F572F612F7708013A031D7C
:100EB4005C2F5D2F612FF7010C30FF2FFF2F0730C0
:100EC400FB007B0886040730FB007B0883160313B2
:100ED4008604FD30FB007B08860502300A128A1165
:100EE400D8250A128A1183120313061C7A2F7B2F2A
:100EF400852FF508031D7F2F802F852FF501F50A17
:100F04000730FF2FFF2F0618882F892F932F75087E
:100F1400013A031D8E2F8F2F932FF5010830FF2FD9
:100F2400FF2F061D962F972FA12FF308031D9B2F2C
:100F34009C2FA12FF301F30A0330FF2FFF2F061973
:100F4400A42FA52FAF2F7308013A031DAA2FAB2F8F
:100F5400AF2FF3010430FF2FFF2F0730FB007B0876
:100F640086040330FB007B08831603138604FB30DE
:100F7400FB007B08860502300A128A11D8250A1262
:100F84008A1183120313061CC82FC92FD32FF40808
:100F9400031DCD2FCE2FD32FF401F40A0530FF2FDC
:100FA400FF2F0618D62FD72FE12F7408013A031DFF
:100FB400DC2FDD2FE12FF4010630FF2FFF2F861CDD
:100FC400E42FE52FEF2FF608031DE92FEA2FEF2F6B
:100FD400F601F60A0930FF2FFF2F8618F22FF32FA0
:100FE400FD2F7608013A031DF82FF92FFD2FF60186
:0C0FF4000A30FF2FFF2F0030FF2F0800F5
:02400E0032FF7F
:00000001FF
